:020000040000FA
:1000000089280230A40036088400340854200630C1
:10001000A5004620A50B09282C202C2029202B08E0
:100020004120A6000430A500A60C2720A50B14280B
:100030002A0841200F392A1A1038A6000530A500D9
:10004000A60C2720A50B2028A40B0C288428031C11
:100050002B282C20462846204620360884000330D2
:10006000A700340880040330A100E8306820340978
:100070008005A703031908000630A100EA306820B4
:100080003128043EA0002019023A080037088400F5
:1000900035088417800484130005A0003508000586
:1000A000200603194E280800FF3A800557288417B8
:1000B00080058428A301A200FF30A207031CA30728
:1000C000031C84280330A100DF3068205C28A101D4
:1000D000E83EA000A109FC30031C7128A00703180A
:1000E0006E28A0076400A10F6E2820187728A01C96
:1000F0007B2800007B2808000310A10CA00CFF3E09
:1001000003187C28200884288313031383126400B7
:100110000800831607309F0009308500FF308600F5
:10012000023087000F30880001309C008312890163
:10013000870188010F300805B80064008A110A128F
:10014000831683101C1B831483128318AA28871517
:100150008A019D2887118A110A12B82064008A1129
:100160000A123D1C9D288A110A1225218A019D2808
:100170000130A3005E308A015B200608BA000F3010
:100180003A05B9003A08A000A10104308A017F2095
:10019000BE000730BE05640005303E028A110A1217
:1001A0000318D92C64003E08013C8A110A12031975
:1001B000E428640002303E028A110A120318D92C86
:1001C0000F30BA053D14080064003908003C8A115C
:1001D0000A12031DED280A30BA0064003908013CF8
:1001E0008A110A12031DF6280B30BA006400390880
:1001F000023C8A110A12031DFF280C30BA00640069
:100200003908033C8A110A12031D08290D30BA006F
:1002100064003908043C8A110A12031D11290E30AA
:10022000BA0064003908053C8A110A12031D1A2914
:100230000F30BA0064003908063C8A110A12031D07
:1002400023291030BA003D1408000F300805B8000B
:1002500064003A08013C8A110A1203199B296400C0
:100260003A08023C8A110A120319CD2964003A089F
:10027000033C8A110A120319012A64003A08043C5B
:100280008A110A120319352A64003A08053C8A11BA
:100290000A120319692A64003A08063C8A110A12F4
:1002A00003199D2A64003A08073C8A110A120319AF
:1002B000D12A64003A08083C8A110A120319052B56
:1002C00064003A08093C8A110A120319392B6400A8
:1002D0003A080A3C8A110A1203196D2B64003A0885
:1002E0000B3C8A110A120319A12B64003A080C3C3A
:1002F0008A110A120319D52B64003A080D3C8A11A1
:100300000A120319092C64003A080E3C8A110A12D9
:1003100003193D2C64003A080F3C8A110A12031994
:10032000712C64003A08103C8A110A120319A52C9A
:100330008A110A12D92C64008A110A123B1CB729AF
:100340003B100730B6000430B4000730B70002306D
:10035000B5003808AB00AA018A0101203808AB00BB
:100360001A30AA008A0101208A110A12CB293B14F3
:100370000730B6000430B4000730B7000230B500D3
:100380003808AB00AA018A0101203808AB001230FE
:10039000AA008A0101203D10080064008A110A1297
:1003A0003C1CEA293C100730B6000430B40007308A
:1003B000B7000230B5003808AB000130AA008A014E
:1003C00001203808AB001A30AA008A0101208A11E6
:1003D0000A12FF293C140730B6000430B40007307D
:1003E000B7000230B5003808AB000130AA008A011E
:1003F00001203808AB001230AA008A0101203D100C
:10040000080064008A110A12BC1C1E2ABC100730A6
:10041000B6000430B4000730B7000230B500380829
:10042000AB000230AA008A0101203808AB001A3064
:10043000AA008A0101208A110A12332ABC1407304B
:10044000B6000430B4000730B7000230B5003808F9
:10045000AB000230AA008A0101203808AB0012303C
:10046000AA008A0101203D10080064008A110A12C6
:100470003C1D522A3C110730B6000430B40007304E
:10048000B7000230B5003808AB000330AA008A017B
:1004900001203808AB001A30AA008A0101208A1115
:1004A0000A12672A3C150730B6000430B400073042
:1004B000B7000230B5003808AB000330AA008A014B
:1004C00001203808AB001230AA008A0101203D103B
:1004D000080064008A110A12BC1D862ABC1107306C
:1004E000B6000430B4000730B7000230B500380859
:1004F000AB000430AA008A0101203808AB001A3092
:10050000AA008A0101208A110A129B2ABC15073011
:10051000B6000430B4000730B7000230B500380828
:10052000AB000430AA008A0101203808AB00123069
:10053000AA008A0101203D10080064008A110A12F5
:100540003C1EBA2A3C120730B6000430B400073013
:10055000B7000230B5003808AB000530AA008A01A8
:1005600001203808AB001A30AA008A0101208A1144
:100570000A12CF2A3C160730B6000430B400073008
:10058000B7000230B5003808AB000530AA008A0178
:1005900001203808AB001230AA008A0101203D106A
:1005A000080064008A110A12BC1EEE2ABC12073031
:1005B000B6000430B4000730B7000230B500380888
:1005C000AB000630AA008A0101203808AB001A30BF
:1005D000AA008A0101208A110A12032BBC160730D7
:1005E000B6000430B4000730B7000230B500380858
:1005F000AB000630AA008A0101203808AB00123097
:10060000AA008A0101203D10080064008A110A1224
:100610003C1F222B3C130730B6000430B4000730D7
:10062000B7000230B5003808AB000730AA008A01D5
:1006300001203808AB001A30AA008A0101208A1173
:100640000A12372B3C170730B6000430B4000730CD
:10065000B7000230B5003808AB000730AA008A01A5
:1006600001203808AB001230AA008A0101203D1099
:10067000080064008A110A12BC1F562BBC130730F5
:10068000B6000430B4000730B7000230B5003808B7
:10069000AB000830AA008A0101203808AB001A30EC
:1006A000AA008A0101208A110A126B2BBC1707309D
:1006B000B6000430B4000730B7000230B500380887
:1006C000AB000830AA008A0101203808AB001230C4
:1006D000AA008A0101203D10080064008A110A1254
:1006E000BB1C8A2BBB100730B6000430B4000730A7
:1006F000B7000230B5003808AB000930AA008A0103
:1007000001203808AB001A30AA008A0101208A11A2
:100710000A129F2BBB140730B6000430B400073018
:10072000B7000230B5003808AB000930AA008A01D2
:1007300001203808AB001230AA008A0101203D10C8
:10074000080064008A110A123B1DBE2B3B110730C2
:10075000B6000430B4000730B7000230B5003808E6
:10076000AB000A30AA008A0101203808AB001A3019
:10077000AA008A0101208A110A12D32B3B150730E7
:10078000B6000430B4000730B7000230B5003808B6
:10079000AB000A30AA008A0101203808AB001230F1
:1007A000AA008A0101203D10080064008A110A1283
:1007B000BB1DF22BBB110730B6000430B40007306C
:1007C000B7000230B5003808AB000B30AA008A0130
:1007D00001203808AB001A30AA008A0101208A11D2
:1007E0000A12072CBB150730B6000430B4000730DE
:1007F000B7000230B5003808AB000B30AA008A0100
:1008000001203808AB001230AA008A0101203D10F7
:10081000080064008A110A123B1E262C3B12073086
:10082000B6000430B4000730B7000230B500380815
:10083000AB000C30AA008A0101203808AB001A3046
:10084000AA008A0101208A110A123B2C3B160730AC
:10085000B6000430B4000730B7000230B5003808E5
:10086000AB000C30AA008A0101203808AB0012301E
:10087000AA008A0101203D10080064008A110A12B2
:10088000BB1E5A2CBB120730B6000430B400073030
:10089000B7000230B5003808AB000D30AA008A015D
:1008A00001203808AB001A30AA008A0101208A1101
:1008B0000A126F2CBB160730B6000430B4000730A4
:1008C000B7000230B5003808AB000D30AA008A012D
:1008D00001203808AB001230AA008A0101203D1027
:1008E000080064008A110A123B1F8E2C3B1307304C
:1008F000B6000430B4000730B7000230B500380845
:10090000AB000E30AA008A0101203808AB001A3073
:10091000AA008A0101208A110A12A32CBB160730F3
:10092000B6000430B4000730B7000230B500380814
:10093000AB000E30AA008A0101203808AB0012304B
:10094000AA008A0101203D10080064008A110A12E1
:10095000BB1FC22CBB130730B6000430B4000730F5
:10096000B7000230B5003808AB000F30AA008A018A
:1009700001203808AB001A30AA008A0101208A1130
:100980000A12D72CBB170730B6000430B40007306A
:10099000B7000230B5003808AB000F30AA008A015A
:1009A00001203808AB001230AA008A0101203D1056
:0609B00008003D100800E4
:020000040000FA
:02400E00713F00
:00000001FF
